:1000000012C0189518951895189518955AC51895F1
:100010001895189518951895189518951895189578
:100020001895189518958FE58DBFC0E6E8E74E2E18
:1000300084E08EBFD3E0F1E05F2EEEEFF3E0A0E6C8
:10004000B0E088278D933197E9F783E389B980E0A1
:1000500080BD88E18AB9662478948B98939A68D693
:1000600084EF81BB80E082BB80EE87BB8FE388BBDF
:1000700083E680936F0083E68093700081E090E0D8
:10008000ABE6B0E08D939C9381E090E0ADE6B0E00C
:100090008D939C93A7E6B0E0E2E3F0E155D68BE1C7
:1000A00080938800A8E8B0E08C91A3E8B0E08D933D
:1000B00088278C93A3E8B0E08FD4E6E3F0E144D640
:1000C000A8E8B0E08C91A9E8B0E08D9388278C93E4
:1000D000A9E8B0E081D4EAE3F0E136D680E090E030
:1000E000A3E9B0E08D939C9380E090E0A8E9B0E0B4
:1000F0008D939C9380E090E0A6E9B0E08D939C9373
:10010000AAE9B0E0E0E4F0E11FD680E08093A5002A
:10011000A3E8B0E06AD475D4A8E8B0E08C9174D4B8
:10012000E6E4F0E168D46DD4A9E8B0E05ED469D427
:1001300019D281E090E0A0E6B0E08D939C93A0E618
:10014000B0E00D911C910E3450E0150714F009F049
:1001500014C04091C40000916F00041709F401C05D
:100160000CC04091B70000917000041709F401C061
:1001700004C0A0E6B0E029D4E2CF8091C40080930F
:100180006F008091B700809370002FD0A8E8B0E096
:100190008C913AD4E2E6F0E12ED46CD4A3EDB0E039
:1001A00024D4E8E6F0E127D465D4AAECB0E01DD46D
:1001B00028D4409180000091C500041709F406C0BE
:1001C000D1D1CED38091C500809380000091B7003B
:1001D0000D3210F009F001C005C08091C1008F7789
:1001E0008093C100A6CF000008950027A6E3B0E0E9
:1001F0008C9184FB0EF401E041E0041709F01AC071
:10020000A7E6B0E04C910091C400041708F402C0C6
:100210006ED00FC00091C400013308F409C00091F2
:1002200095000F3F08F002C0BDD001C005D001C04D
:1002300003D001C0F4D0089588E0E3EDF0E001E0E0
:100240000A93A2E6B0E0E6D680E090E0A1E7B0E055
:100250008D939C9321D187E0E3EDF0E001E00A93D8
:10026000A2E6B0E0D7D681E090E0A1E7B0E08D93C0
:100270009C9312D185E0E3EDF0E001E00A93A2E661
:10028000B0E0C8D682E090E0A1E7B0E08D939C9307
:1002900003D184E0E3EDF0E001E00A93A2E6B0E0F0
:1002A000B9D683E090E0A1E7B0E08D939C93F4D0C1
:1002B00082E0E3EDF0E001E00A93A2E6B0E0AAD626
:1002C00084E090E0A1E7B0E08D939C93E5D081E0DD
:1002D000E3EDF0E001E00A93A2E6B0E09BD685E012
:1002E00090E0A1E7B0E08D939C93D6D0089588E08C
:1002F000EAECF0E001E00A93A2E6B0E08BD680E001
:1003000090E0A1E7B0E08D939C93C6D087E0EAEC43
:10031000F0E001E00A93A2E6B0E07CD681E090E054
:10032000A1E7B0E08D939C93B7D085E0EAECF0E0D4
:1003300001E00A93A2E6B0E06DD682E090E0A1E78A
:10034000B0E08D939C93A8D084E0EAECF0E001E06B
:100350000A93A2E6B0E05ED683E090E0A1E7B0E0C9
:100360008D939C9399D082E0EAECF0E001E00A934F
:10037000A2E6B0E04FD684E090E0A1E7B0E08D9334
:100380009C938AD081E0EAECF0E001E00A93A2E6D7
:10039000B0E040D685E090E0A1E7B0E08D939C937B
:1003A0007BD0089585E0E9E7F0E001E00A93A2E65A
:1003B000B0E030D680E090E0A1E7B0E08D939C9370
:1003C0006BD084E0E9E7F0E001E00A93A2E6B0E058
:1003D00021D681E090E0A1E7B0E08D939C935CD0C2
:1003E00082E0E9E7F0E001E00A93A2E6B0E012D68D
:1003F00082E090E0A1E7B0E08D939C934DD081E046
:10040000E9E7F0E001E00A93A2E6B0E003D683E07A
:1004100090E0A1E7B0E08D939C933ED0089584E0F6
:10042000EAE9F0E001E00A93A2E6B0E0F3D582E069
:1004300090E0A1E7B0E08D939C932ED083E0EAE9B1
:10044000F0E001E00A93A2E6B0E0E4D583E090E0BA
:10045000A1E7B0E08D939C931FD082E0EAE9F0E041
:1004600001E00A93A2E6B0E0D5D584E090E0A1E7F0
:10047000B0E08D939C9310D081E0EAE9F0E001E0D8
:100480000A93A2E6B0E0C6D585E090E0A1E7B0E02F
:100490008D939C9301D00895A3E9B0E096D2A2E693
:1004A000B0E08C91AAE6B0E08C9394E0AAE6B0E0CC
:1004B00050D4A1E7B0E08C91A5E3B0E06BD460D458
:1004C0000C900822689409F4E894882780F98095B4
:1004D00080FBA1E7B0E08C91A5E3B0E05BD450D401
:1004E0000C9016F0092201C0082A0C92AAE6B0E08E
:1004F0008C9182BBABE6B0E08D919C9192D2A3E946
:10050000B0E00D911C910D3750E0150709F007C0C0
:10051000E6D080E090E0A3E9B0E08D939C93A1E762
:10052000B0E08C91A5E3B0E035D42AD40C90082239
:10053000689409F4E894882780F9809580FBA1E706
:10054000B0E08C91A5E3B0E025D41AD40C9016F05D
:10055000092201C0082A0C92ADE6B0E08D919C9171
:1005600060D2089582E0E0E367D463E382E0E0E3F1
:10057000BB27A6E121E02A938BD4BB27A6E182E02A
:10058000E0E321E02A93AAD4A5E9B0E05C930091CE
:1005900095000F3F09F001C0089582E0E0E34CD4DC
:1005A0006CEC82E0E0E3BB27A6E121E02A9370D463
:1005B00064E482E0E0E3BB27A6E121E02A9368D46B
:1005C00082E0E0E339D46CEC82E0E0E3BB27A6E113
:1005D00021E02A935DD46EEB82E0E0E3BB27A6E145
:1005E00021E02A9355D481E0809376000091760033
:1005F000023010F009F017C0BB27A6E182E0E0E36B
:1006000021E02A936BD4A6E7B0E0AD90BB24A2E72B
:10061000B0E0AA0DBB1D5C93A6E7B0E08C918F5FA4
:100620008C9308F4E3CFA3E7B0E08C91A7E7B0E0A8
:100630008D9388278C93A7E7B0E08D919C91A7E7D5
:10064000B0E08D939C9300917400003010F009F09D
:1006500001C007C080E090E0A7E7B0E08D939C93D5
:1006600004C091E0A7E7B0E07CD30091730041E0C3
:100670000423AFE7B0E00C9300917F00013009F054
:1006800006C0A0E9B0E0ECE6F0E15ED305C0A0E969
:10069000B0E0E0E7F0E158D3A9E7B0E0E7E7F0E049
:1006A00060D4A9E7B0E098D1E4E7F0E14DD3E0E908
:1006B000F0E0A9E7B0E090D1A8D4A8E8B0E08C9130
:1006C000A3D1E6E7F0E197D1ECE7F0E194D1A9E717
:1006D000B0E08BD1EAE8F0E18ED193D10895002704
:1006E000A6E3B0E08C9184FB0EF401E041E0041736
:1006F00009F0B0C00027A6E3B0E08C9180FB0EF4B7
:1007000001E040E0041709F03DC00091A500013070
:1007100009F008C088B390E2892788BB80E0809305
:10072000A50008950027A6E3B0E08C9183FB0EF4AA
:1007300001E041E0041709F013C0A6ECB0E08C9191
:100740008F5F8C930091C600073110F009F001C053
:1007500003C080E08093C60080E08093C40012C094
:1007600087E38093C400A7ECB0E08C918F5F8C93FB
:100770000091C7000F3110F009F001C003C081E003
:100780008093C7000027A6E3B0E08C9181FB0EF4B4
:1007900001E040E0041709F030C00027A6E3B0E014
:1007A0008C9183FB0EF401E041E0041709F013C0C3
:1007B000A5ECB0E08C918F5F8C930091C5000B335A
:1007C00010F009F001C003C080E08093C50080E014
:1007D0008093C40012C087E38093C400A8ECB0E00B
:1007E0008C918F5F8C930091C8000C3010F009F051
:1007F00001C003C081E08093C8000027A6E3B0E0F9
:100800008C9182FB0EF401E040E0041709F021C056
:100810000027A6E3B0E08C9183FB0EF401E041E0F9
:10082000041709F004C080E08093C40012C087E37D
:100830008093C400A9ECB0E08C918F5F8C93009101
:10084000C900033610F009F001C003C080E08093B6
:10085000C90085C00027A6E3B0E08C9180FB0EF4B0
:1008600001E040E0041709F024C00027A6E3B0E04F
:100870008C9183FB0EF401E041E0041709F019C0EC
:10088000A6E9B0E0A2D0A6E9B0E00D911C91073135
:1008900050E0150714F009F001C006C080E090E0B8
:1008A000A6E9B0E08D939C93AFE9B0E0E6E9F0E013
:1008B00058D30027A6E3B0E08C9181FB0EF401E051
:1008C00040E0041709F024C00027A6E3B0E08C91B3
:1008D00083FB0EF401E041E0041709F019C0A8E918
:1008E000B0E073D0A8E9B0E00D911C910B3350E05B
:1008F000150714F009F001C006C080E090E0A8E9F7
:10090000B0E08D939C93A2EAB0E0E8E9F0E029D34F
:10091000E2EAF0E0A0E6B1E078D3E0E6F1E0A2EAB6
:10092000B0E01127222702E033273AD2EFE9F0E0C6
:10093000A0E6B1E06AD3E0E6F1E0AFE9B0E011276C
:10094000222702E033272CD2EFE9F0E0AAE9B0E059
:100950005CD3E2EAF0E0AAE9B0E03ED056D30895D5
:10096000A6E9B0E00D911C91003050E0150709F0A8
:100970000AC0A8E9B0E00D911C91003050E01507C5
:1009800009F001C00895A6ECB0E04D915527A6E905
:10099000B0E00D911C910417150709F013C0A5ECE8
:1009A000B0E04D915527A8E9B0E00D911C910417D6
:1009B000150709F007C088B390E2892788BB81E05A
:1009C0008093A5000895F894FFCFED91FC91EF5F1F
:1009D000FF4FFC93EE9308958F938D918823E9F751
:1009E00011978F910895A0E6B1E08D91882311F0C1
:1009F0000BD0FBCF0895C0D1802D11F005D0FBCFD7
:100A000008958DE001D08AE05D9BFECF8CB90895FA
:100A10003197F1F70895689462F80895E89462F8C0
:100A20000895EF93FF93EE27E82BE92B31F0E0EAEE
:100A3000FFE03197F1F70197D1F7FF91EF9108951A
:100A400089B78F7E89BF80E08FBD8AE08EBD80E050
:100A500090E090934D0080934C0080E593EC909350
:100A60004B0080934A0088B7806188BF89B7806156
:100A700089BF089525D0AAECB0E0E7ECF0E013D0F0
:100A8000339702C0EDE0FF2782814AD28AE38D933B
:100A9000818146D28AE38D93808142D288278C93CC
:100AA0000895EDE0FF2780813BD28EE28D93818116
:100AB00037D28EE28D93828133D288278D93089529
:100AC0000895FF93EF936F938F939F937F938FB7C7
:100AD0008F93E6EBF0E0638564FD3FC07081739512
:100AE000708380B366FF02C098E0892783FB80F99A
:100AF000862780FF32C060F98827808346F0E8941B
:100B0000763008F0689436D08287718726C07633B5
:100B1000E0F09927918362FF20C0958796878281B4
:100B200087878381808B8481818B8581828B86817D
:100B3000838B8781848760686B7F638780858874F7
:100B400081F463FDEFD0AAD00CC0918193959B33C3
:100B500011F4808586FF6B7F91835ED063870EF4EE
:100B6000D5D08F918FBF7F919F918F916F91EF9192
:100B7000FF91189571858285918116F473957D7F1B
:100B8000869587F98287943129F4808777270EF03C
:100B9000706808959C3119F430D0828338C0933244
:100BA00019F429D0838333C0993219F423D0848374
:100BB00008959C3229F482958695877087830895DD
:100BC000913319F416D085830895993319F416D00A
:100BD000868308959A3361F41AD051F486A18395DF
:100BE0008C3309F48827928196A3891709F46460ED
:100BF0000895869586958F7786958F7784FD8650A4
:100C000085FD8C5086FD885187FD8053089570FBCB
:100C1000769577F9707F0895E89485858395858723
:100C2000883208F408958827858786858395868786
:100C30008C33A0F1772776878785839587878130E6
:100C400009F468948C3350F1778780898395808B81
:100C5000883120F1708B81898395818B8D31F0F003
:100C600092898F3111F080F408C0943069F0963089
:100C700059F0993049F09B3039F0923079F473890A
:100C8000737011F48E3150F071E0718B9395928BEB
:100C90009D3020F0728B83898395838B0F921F92F6
:100CA0002F923F924F925F927F92AF92BF920F939B
:100CB0001F932F933F934F935F936F937F938F93E4
:100CC0009F93AF93BF93CF93DF93EF93FF938FB730
:100CD0008F9389DA8F918FBFFF91EF91DF91CF9141
:100CE000BF91AF919F918F917F916F915F914F9144
:100CF0003F912F911F910F91BF90AF907F905F9088
:100D00004F903F902F901F900F900895E6EBF0E0EA
:100D100063856F7E68606387BF93AF9391DEAF9109
:100D2000BF910895E6EBF0E0638560616387089505
:100D300088278093C100EACF7091BE00882775FB99
:100D400080F974FB81F9089517D00D920020E1F726
:100D50000895903029F08C91880F9A95E9F78C933B
:100D60000895903041F00D911C91169507959A9534
:100D7000E1F71C930E930895C895319600200895CD
:100D800091E0882321F08894991F8A95E9F7892FAB
:100D900090950895883018F011968850FBCF0895EB
:100DA0002E2E3F2E992781918D3209F0939588231D
:100DB000D1F79A95E22DF32D112361F0091718F060
:100DC00011F0101B01C0191B28F021F080E28D9357
:100DD0001A95E9F780818D3219F48D93319604C00C
:100DE000222311F08BE28D93091738F031F0091BA3
:100DF00021F080E38D930A95E9F781918D93882303
:100E0000E1F7332351F0EA2FFB2F319633958E9182
:100E100082933A95E1F78EE28C9308950181082B35
:100E20000183128119231283EF93FF93E4E0F0E032
:100E3000EFDDFF91EF910895EEDDFF27A1DFEEDFFB
:100E4000EF93FF93ECE7F7E0E3DDFF91EF91182BD1
:100E5000128309230183EF93FF93E4E6F1E0D8DDE9
:100E6000FF91EF911081182359F4EF93FF93ECE772
:100E7000F7E0CEDDFF91EF911081182309F0CEDD70
:100E8000EF93FF93ECE7F7E0C3DDFF91EF91089557
:100E900077DFFF2729915D9148E0C0DFEF93FF9353
:100EA000E4E0F0E0B5DDFF91EF91579510F4182BD9
:100EB0001283EF93FF93ECEEF0E0AADDFF91EF9148
:100EC000182B1283EF93FF93E4E0F0E0A1DDFF9194
:100ED000EF914A9511F72A95F1F6089551DFFF2712
:100EE000299148E055279ADF09230183EF93FF9367
:100EF000E4E1F0E08DDDFF91EF91889410811823FB
:100F000009F008945795EF93FF93E0EBF0E080DD54
:100F1000FF91EF914A9539F75D932A9511F708955E
:100F200000278A3018F08A500395FBCF005D0D939F
:100F3000805D8D930895000F111F221F331F0895A8
:100F400000951095209530950F5F1F4F2F4F3F4F05
:100F50000895019110810EC001911191219130816C
:100F60000BC00191108117FF05C03FEF2FEF04C0A8
:100F7000008111272227332737FF03C0E1DF8DE2ED
:100F80008D93CF93DF93CF92DF92EF92AA24BB246D
:100F9000CC24DD24EE2440E2CAE0DD2755E093E3D3
:100FA0008881890F87FD9F7083FD907F891B8993BE
:100FB0005A95A9F7C0DFAA1CBB1CCC1CDD1CEE1C7B
:100FC0004A9551F7E894EFE0FF2782910ED0EB307D
:100FD000E0F71EF068948A2D0CD088278D93EF904F
:100FE000DF90CF90DF91CF910895982F829501D017
:100FF000892F8F70805D26F0803309F408956894FE
:101000008D93089588278D93089581918D938823DA
:10101000E1F7089509919191992351F08A95D9F7B3
:10102000319781918D930A9519F08823D1F708950E
:10103000E9CF353500005B324A005B3F32356C004A
:101040003030303000004443462D37372055687229
:1010500020563234206675657220494E2D3132415A
:1010600000005B333B3166002D2D00003530000061
:10107000303000002C005B353B31660054656D70EC
:0E108000657261747572203A200020430000F2
:00000001FF
